:100000000C94BD020C94DA020C94F5020C94DA0202
:100010000C94DA020C94DA020C94DA020C94DA02F0
:100020000C94DA020C94DA020C9417210C94DA0284
:100030000C94DA020C94DA020C94DA020C94DA02D0
:100040000C94DA020C94DA020C94DA020C94DA02C0
:100050000C94DA02A607A607D207D2073A08650968
:10006000650965095808F108020902090000000045
:10007000000000000000000000002C00E600E70087
:10008000500051004F003C000000E000E300E2009F
:100090002C00015123000000110010003600370031
:1000A0003800E50052000000E1001D001B000600C2
:1000B0001900050000000B000D000E000F003300BA
:1000C0003400280000003900040016000700090071
:1000D0000A00000018000C00120013002F0030006E
:1000E000310000002B0014001A0008001500170052
:1000F000000024002500260027002D002E002A00E5
:10010000000029001E001F00200021002200000026
:100110001C000000000000000000000000000000C3
:1001200000000000000000000000000000000100CE
:1001300001000100010001000100010000000100B8
:1001400001000100010001003F000000010001006A
:100150000100010001000100010000000100010098
:100160000100010001000100000001000100010088
:100170000100010001000100000001000100010078
:100180000100010001000000010001000100010068
:100190000100010001000000010001000100010058
:1001A0000100010000004000410042004300440003
:1001B00045000100000001003A003B003C003D000A
:1001C0003E000000010000000000000000000000F0
:1001D000000000000000000000000000000000001F
:1001E0000000010001000100010001000100010008
:1001F00000000100010001000100010001000000F9
:1002000001000100010001000100010001000000E7
:1002100001000100010001000100010000000100D7
:1002200001000100010001000100010000000100C7
:1002300001000100010001000100000001000100B7
:1002400001000100010001000100000001000100A7
:100250000100010001000100000001000100010097
:100260000100010001000100000001000100010087
:10027000010001000100000001000000000000007A
:10028000000000000000000000047F3F1F643214E3
:10029000643214783C1E1E140A05222325262829C0
:1002A0002A2C2D2F3032333536383A3B3D3E4042F2
:1002B000434547494A4C4E5051535557595A5C5E35
:1002C0006062646668696B6D6F71737577797B7D49
:1002D0007F81838587898A8C8E90929496989A9C48
:1002E0009E9FA1A3A5A7A8AAACAEAFB1B3B4B6B860
:1002F000B9BBBCBEBFC1C2C3C5C6C7C9CACBCCCDC2
:10030000CED0D1D2D2D3D4D5D6D7D7D8D9D9DADA9C
:10031000DBDBDBDCDCDCDCDCDDDDDDDDDCDCDCDC1C
:10032000DCDBDBDBDADAD9D9D8D7D7D6D5D4D3D250
:10033000D2D1D0CECDCCCBCAC9C7C6C5C3C2C1BF2E
:10034000BEBCBBB9B8B6B4B3B1AFAEACAAA8A7A592
:10035000A3A19F9E9C9A98969492908E8C8A89874E
:100360008583817F7D7B79777573716F6D6B69682C
:10037000666462605E5C5A5957555351504E4C4A00
:100380004947454342403E3D3B3A383635333230AB
:100390002F2D2C2A292826252322FFAA7F5540000D
:1003A0000101010101010101010202020202020236
:1003B0000202030303030303030304040404040409
:1003C00004050505050506060606060707070707CF
:1003D00008080808090909090A0A0A0B0B0B0C0C82
:1003E0000C0D0D0D0E0E0E0F0F0F1010111111121E
:1003F0001213131414151516161717181819191A9D
:100400001A1B1B1C1D1D1E1E1F20202122222324FF
:1004100024252626272829292A2B2C2D2D2E2F303E
:10042000313232333435363738393A3B3C3D3E3F52
:10043000404142434445464748494A4C4D4E4F503F
:10044000515354555658595A5B5D5E5F61626465FD
:100450006668696B6C6D6F7072737577787A7B7D87
:100460007E8082838587888A8C8E8F9193959698DB
:100470009A9C9EA0A2A3A5A7A9ABADAFB1B3B5B7F7
:10048000BABCBEC0C2C4C6C9CBCDCFD1D4D6D8DBCE
:10049000DDDFE2E4E7E9EBEEF0F3F5F8FAFDFF0962
:1004A000023B00020100A0FA09040000010301015F
:1004B0000009210101000122400007058103080015
:1004C00001090401000103000000092101010001EC
:1004D0002232000705830308000112011001000009
:1004E00000084D5964530002010200010A03530041
:1004F00050003600340000000A0359004D0044004B
:100500004B0000000403090405010980A1018503D3
:1005100019012AB700150126B70095017510810051
:10052000C0050C0901A101850419012AA0021501C9
:1005300026A002950175108100C005010906A101E0
:10054000050719E029E715002501950875018102C5
:100550009501750881030507190029FF150026FF7D
:10056000009506750881000508190129059505758E
:10057000019102950175039103C011241FBECFE5BF
:10058000D8E0DEBFCDBF11E0A0E6B0E0ECE9FAE4D0
:1005900002C005900D92AE30B107D9F723E0AEE06E
:1005A000B1E001C01D92A530B207E1F70E943714F7
:1005B0000C944C250C940000A82FB92F80E090E0FB
:1005C00041E050EA609530E009C02D91822797956F
:1005D000879510F084279527305EC8F36F5FA8F3E6
:1005E0000895EADF8D939D930895CF93CFB7CF936E
:1005F000C395839BE9F7839B0EC0839B0CC0839BB1
:100600000AC0839B08C0839B06C0C091DC02C395CF
:10061000C093DC02A6C0DF93C091DB02DD27CD5181
:10062000DD4F839B02C0DF91E6CF2F930F931F9383
:1006300000B32FEF03FB20F94F933F9310B34FEF1D
:10064000012703FB21F93BE031C04E7F012F10B39E
:10065000216028C0102F4D7F2260000000B329C008
:100660004B7F2460012F000010B32BC010B3477FD5
:1006700028602AC04F7E00B320612CC04F7D10B38C
:1006800020622FC04F7B00B3206432C0422700B3EA
:1006900049934FEF0000102713FB20F910B31C7093
:1006A000C9F1297F91F2012703FB21F900B3237FD0
:1006B00089F2315058F1102713FB22F910B3277E2D
:1006C00079F2012703FB23F92F7C81F200B3102775
:1006D00013FB24F92F7971F200C010B3012703FB3B
:1006E00025F92F7359F200C000B3102713FB26F928
:1006F000223040F200C010B3012703FB27F9243059
:1007000028F64F77206810B30000F9CF10E81ABF21
:1007100000271CC03B503195C31BD04010E81ABFC6
:100720000881033C11F10B3401F12091D8021981A9
:10073000110F1213EDCF4A81441F093669F10D32B2
:1007400011F0013E29F74F7009F0042F0093E102E8
:100750003F914F911F910F912F91DF91CAB7C7FD24
:1007600047CFCF91CFBFCF9118952091E10222239F
:1007700079F31091DF02112309F044C034300AF4F8
:1007800043C03093DF022093DA021091DB023BE09A
:10079000311B3093DB0238C00091DF02013094F549
:1007A0000AE54F7049F43091860034FD2FC0009364
:1007B0008600C5EBD2E02EC0433059F0443091F0B2
:1007C0003091C00234FD22C00093C002C1ECD2E0DF
:1007D00021C03091F90234FD19C00093F902CAEF2B
:1007E000D2E018C03091CC0234FD10C00093CC028E
:1007F000CDECD2E00FC02795A8F45150A9F4220FF8
:100800000000F9CF4AE503C042ED01C0432FC4E127
:10081000D0E032E011B31C60939A11BB02B320E424
:100820001CE05F93012756E002BB279520F451504E
:1008300021F4220FF9CF012756E000003B5A02BBFA
:10084000D0F2279528F4515029F4220F0000F9CF57
:10085000012756E0279502BB20F4515021F4220FC6
:10086000F9CF012756E02991332302BB21F6037FFC
:100870001091E002110FC651D04002BB11F010934D
:10088000D80210E81ABF086011B3137F402F437FCE
:100890005F9100C000C002BB11BB42BB59CF08959D
:1008A0000C944F040C9450040C944F048FEF87BBAE
:1008B00088BB1ABA94B39B7B94BB8F988BBB85B3D0
:1008C0008C6F85BB979A0E941E0590E09093610003
:1008D00080936000EDE1F1E0A1E1B1E011921192AD
:1008E0001D921D9281E0E932F807C1F786E00E946F
:1008F000F6130C94D2057F928F929F92AF92BF9283
:10090000CF92DF92EF92FF920F931F93CF93DF93DB
:1009100000D01F92CDB7DEB780916000909161004A
:10092000892B71F0809110018F5F809310018111EC
:1009300007C00E941E0590E09093610080936000C4
:1009400031E1C32E31E0D32EE12CF12CB12C42E168
:10095000A42E88248394912C6FE7762EA98284019B
:100960000E2C01C0000F0A94EAF7102F10951A837D
:1009700024E630E042E050E0BE016F5F7F4F80E44C
:100980000E94C11F909361008093600007BB18BB59
:1009900009B3009510E0798224E630E041E050E0B0
:1009A000BE016F5F7F4F80E40E94E71F898190E066
:1009B000809590958F7799279695982F882797956A
:1009C0008795802B912BF601208131818217930727
:1009D00021F091838083BB24B394FFEFEF1AFF0AC9
:1009E00082E0C80ED11CE6E0EE16F10409F0B6CFA5
:1009F0002B2D46E06DE171E081E191E00E94F7135B
:100A00000E94D4058B2D0F900F900F90DF91CF9106
:100A10001F910F91FF90EF90DF90CF90BF90AF901C
:100A20009F908F907F900895E82FF0E0EE0FFF1FCA
:100A3000E35EFE4F80819181089508951F93CF93C7
:100A4000DF9300D01F92CDB7DEB78FEF9FEF90936B
:100A50006100809360008091290181110EC00E9485
:100A6000CA1E81E0809329012FEF8EE994E2215084
:100A700080409040E1F700C0000019821A821FEF09
:100A80001B8324E630E043E050E0BE016F5F7F4F00
:100A900080E40E94C11F9093610080936000892BC5
:100AA00031F58CE089831A821B8324E630E043E031
:100AB00050E0BE016F5F7F4F80E40E94C11F9093A2
:100AC000610080936000892B91F484E189831A830B
:100AD0001B8324E630E043E050E0BE016F5F7F4FB0
:100AE00080E40E94C11F9093610080936000809118
:100AF00060000F900F900F90DF91CF911F9108959C
:100B000081E0089581E008950C94820508950C9485
:100B100086051F93CF93DF9300D000D01F92CDB7EF
:100B2000DEB749835A836B8330912B0189819A8187
:100B3000311114C0662359F0222349F00E949E0B04
:100B4000182F682F89819A810E94470B03C00E9449
:100B5000720B182F69817A81812F04C00E949E0B2D
:100B600069817A810F900F900F900F900F90DF9115
:100B7000CF911F910C94C612FC01262F4081518108
:100B80006281738184810C94890581E00895CF93FB
:100B9000DF93EC0160E00E94BC05BE01DF91CF91C4
:100BA0000C9487050C9452040C94540408950E94EC
:100BB000F1090E94D6052FEB87E299E02150804091
:100BC0009040E1F700C000000C943D210F931F936B
:100BD000CF93DF938C0161E00E94BC05EC01B8016A
:100BE0000E948405882309F444C0B801CE010E9404
:100BF000781E8823F1F1B801CE010E94A41B88233E
:100C0000C1F1B801CE010E94D41D882391F1B80131
:100C1000CE010E94B71A882361F1F80182818823EE
:100C200009F1CB358DE5D807C1F050F4C115FCE5CD
:100C3000DF0781F0CF3DDC45A9F40E94D51019C033
:100C4000CC35EDE5DE0761F0CD35DD4559F40E9488
:100C5000181008C00E94D7050CC00E94211002C0C5
:100C60000E942410C801DF91CF911F910F910C9425
:100C7000800580E0DF91CF911F910F9108950E9430
:100C8000C1200E945C060C9434190E945F060E94E9
:100C9000001A0C94C72008950C944B0681E0089527
:100CA0000C944E060895CF93C82F0E944C068C2FAB
:100CB0000E945006CF91089580E00C9453060E9444
:100CC0002E200C9453060E942E2090912A01891701
:100CD00021F080932A010C9453060895CF93DF935B
:100CE000CDB7DEB72B970FB6F894DEBF0FBECDBFE2
:100CF0004F83588769877A878B8761110E94640FB9
:100D00009E012F5F3F4F86E0F90111928A95E9F726
:100D100085E0FE013796D90101900D928A95E1F7A1
:100D200089819A814C815D81452B31F09F3F31F45F
:100D300091E08F3F19F403C091E001C090E090FF73
:100D400009C049815A816B817C818D819E810E947D
:100D5000850E05C0C9010E94C5058111F2CF2B96F1
:100D60000FB6F894DEBF0FBECDBFDF91CF910895CF
:100D7000FC01808191810E94E00B0895CF9388232C
:100D800009F44DC0C82F8CEF8C0F813AF8F48C2FEA
:100D90000E94981D811143C06C2F80916400909136
:100DA00065000E947D20882349F06C2F80916400AB
:100DB000909165000E94B5200E94860F6C2F809153
:100DC0006400909165000E94B3200CC080E28C0FFB
:100DD000883058F4C77081E001C0880FCA95EAF7DF
:100DE0000E94470FCF910C94860FEBE5EC0FE33098
:100DF00040F4F0E0EB54FF4F808190E0CF910C94F1
:100E00004520C85AC73158F4EC2FF0E0EE0FFF1F11
:100E1000E957FF4F80819181CF910C945B20CF9156
:100E20000895882349F1682F8CEF860F813A38F4B2
:100E300080916400909165000E94B5200CC080E212
:100E4000860F883050F4677081E001C0880F6A9582
:100E5000EAF70E944D0F0C94860F8BE5860F8330C6
:100E600020F480E090E00C944520685A673120F42B
:100E700080E090E00C945B2008951F93CF93DF9364
:100E8000182FEB010E94BE06209741F087EB9BE0F4
:100E90000197F1F700C000002197F6CF812FDF9175
:100EA000CF911F910C941107893319F060E070E025
:100EB00002C060E570E00C943D07882321F00E9499
:100EC000470F0C94860F0895882321F00E944D0F40
:100ED0000C94860F0895CF92DF92EF92FF920F93BA
:100EE0001F93CF93DF937C01D62FC72FFC01128174
:100EF000058102950F700E943D0F8823B9F01123E0
:100F0000A9F08C2F807F803421F080E28D0F883013
:100F100068F08091870282FD09C082E00E94E60F9E
:100F20000E943D0F91E0D82ED92601C0D12CCC2EA5
:100F3000C2948FE0C8228C2D90E08C30910508F08F
:100F4000C4C1FC01E65DFF4F0C949B248C2F807F75
:100F5000CF70882311F0C295C07F112399F0CC2364
:100F600009F49FC180E28D0F883010F0D11104C0C8
:100F70008C2F0E94470F03C08C2F0E94570F0E9496
:100F8000860F8FC18D2F0E941107CC2309F49DC1BC
:100F900080E28D0F883038F1DD2329F18C2F0E94FB
:100FA0005D0F24C08C2F807FCF70803211F0C295EE
:100FB000C07FDD2319F0D130A1F13DC080918702BF
:100FC00082FF17C0112349F0CC2329F08C2F0E94F7
:100FD000470F0E94860F80E065C180E00E941107E4
:100FE000CC2309F472C18C2F0E944D0F0E94860FF2
:100FF0006CC1112371F0002341F0013031F40E94E3
:10100000670F8C2B0E946F0F60C10E94670F8C2BA3
:101010001DC0002319F0013009F457C10E947C0F54
:1010200025C0112321F0063008F04FC10EC0053055
:1010300008F04BC11BC0112361F0002331F0F70110
:10104000858180FF2EC18F7085838C2F0E945D0764
:101050003CC1002359F0D93309F034C1FFEF0DEE44
:1010600012E0F15000401040E1F72AC18C2F0E949D
:1010700064072BC18C2F86958695837019F081307B
:1010800061F023C1112321F08D2F9C2F937002C09A
:1010900080E090E00E94452020C1112321F08D2F97
:1010A0009C2F937002C080E090E00E945B2015C1ED
:1010B0008C2F837009F047C011110BC12D2F229581
:1010C00026952770220F220F6D2F6F70862F90E0CC
:1010D000A0E0B0E0022E04C0880F991FAA1FBB1F1A
:1010E0000A94D2F7D4FF10C04FE050E060E070E007
:1010F00004C0440F551F661F771F2A95D2F74095ED
:1011000050956095709503C040E050E0BA01C695D7
:10111000C695C3708A019B01082B192B2A2B3B2BE8
:10112000C901B801C23049F058F4C13019F00E9429
:101130005D0ACFC00E944B0ACCC00E946F0AC9C092
:101140000E94490AC6C0112319F08C2F817001C07A
:101150008695882309F4BDC02D2F229526952770EA
:10116000220F220F6D2F6F70862F90E0A0E0B0E06D
:10117000022E04C0880F991FAA1FBB1F0A94D2F722
:10118000D4FF10C04FE050E060E070E004C0440FB6
:10119000551F661F771F2A95D2F740955095609589
:1011A000709503C040E050E0BA01C695C695C37083
:1011B0008A019B01082B192B2A2B3B2BC901B80153
:1011C000C23049F058F4C13019F00E94220B81C09E
:1011D0000E94100B7EC00E94340B7BC00E94830AC9
:1011E00078C0CF70112339F08C2F0E94A90A8D2F5F
:1011F0000E945D076EC08D2F0E9464078C2F0E9495
:10120000CA0A67C0D23F21F128F4D03F41F0D13F54
:10121000C1F043C0D33F19F1D43F79F03EC0112350
:1012200041F0053008F051C08C2F8F710E94EF0AF9
:101230004CC0063008F049C0F7CF8091870282FF8A
:1012400018C0112339F08C2F8F710E94A90A3DC05C
:101250001123C9F38C2F8F710E94CA0A36C0112343
:1012600029F08C2F8F710E94940A2FC00E948F0A40
:101270002CC0112349F0CF718C2F0E94A90A63E082
:101280008C2F0E94CB0F21C081E00E94E60F02301C
:10129000E0F082E00E94E60F18C0112331F0002335
:1012A00091F28D2F0E94BE0610C0002399F2D9330F
:1012B00049F41FEF2DEE32E0115020403040E1F7AD
:1012C00000C000008D2F0E94110788EF8C0D843024
:1012D00020F40E942E200E945306DD20C9F00E94B7
:1012E000390F80FD15C0F70112820E94330F0E9452
:1012F000A90AC7010E94A9090E94330FDF91CF916B
:101300001F910F91FF90EF90DF90CF900C94CA0A3D
:10131000DF91CF911F910F91FF90EF90DF90CF90D1
:1013200008950F931F93CF93DF93EC016881798128
:101330008A810E94EB0B8C010E94460B0E94370AA7
:10134000B801CE010E946B07DF91CF911F910F91E1
:101350000895CF93DF93EC01988189812B813C81A3
:10136000232B31F08F3F31F481E09F3F19F403C00C
:1013700081E001C080E080FD1DC0CE010E94E60535
:10138000811110C00E943D0F8823A1F08A8188231B
:1013900089F08091870282FD0DC082E0DF91CF91BC
:1013A0000C94E60FCE010E949109CE01DF91CF91FE
:1013B0000C94C705DF91CF91089580E090E00E94E2
:1013C000452080E090E00E945B200E94640F0C9416
:1013D000860F80916400909165000E94B7200C9464
:1013E000DD090E94540F0C94E90992959F70963084
:1013F00079F010F4925001C09A50923068F4803F16
:1014000069F018F4883E40F409C0843F29F406C00E
:10141000883E20F0813F11F080E0089581E008953A
:10142000FC01808191810E94E00B0E94F5090895E2
:10143000CF93DF9300D000D01F92CDB7DEB70F90CF
:101440000F900F900F900F90DF91CF910895CF9351
:10145000DF9300D000D000D0CDB7DEB726960FB610
:10146000F894DEBF0FBECDBFDF91CF9108950895F0
:1014700008950C94380A0C94390A0E943B0A609330
:101480006C0170936D0180936E0190936F010C94C9
:10149000DD090C943D0A0F931F9300916C0110918C
:1014A0006D0120916E0130916F01602B712B822BA9
:1014B000932B1F910F910C943D0A0F931F93009152
:1014C0006C0110916D0120916E0130916F016023CC
:1014D0007123822393231F910F910C943D0A0F9344
:1014E0001F9300916C0110916D0120916E0130915C
:1014F0006F0160277127822793271F910F910C940A
:101500003D0A0C94380A0E94810A60936801709326
:10151000690180936A0190936B010C94DD0960E08E
:1015200070E0CB010C94830A0F931F9341E050E0CD
:1015300060E070E08A019B0104C0000F111F221FB0
:10154000331F8A95D2F7C901B8011F910F910C94EE
:10155000830A0F931F9341E050E060E070E004C005
:10156000440F551F661F771F8A95D2F78091680137
:1015700090916901A0916A01B0916B018A019B0170
:10158000082B192B2A2B3B2BC901B8011F910F9156
:101590000C94830A0F931F9341E050E060E070E0E9
:1015A00004C0440F551F661F771F8A95D2F74095D8
:1015B0005095609570958091680190916901A09116
:1015C0006A01B0916B018A019B01082319232A2328
:1015D0003B23C901B8011F910F910C94830A0F930B
:1015E0001F9341E050E060E070E004C0440F551FDD
:1015F000661F771F8A95D2F78091680190916901E3
:10160000A0916A01B0916B018A019B0108271927FB
:101610002A273B27C901B8011F910F910C94830A17
:101620000F931F93009168011091690120916A0145
:1016300030916B01602B712B822B932B1F910F919B
:101640000C94830A0F931F93009168011091690114
:1016500020916A0130916B016023712382239323CF
:101660001F910F910C94830A0F931F9300916801AF
:101670001091690120916A0130916B0160277127F7
:10168000822793271F910F910C94830A08952FE0CE
:10169000929F800D1124E82FE695E695E6958770D8
:1016A00051E001C0550F8A95EAF785E0E89FF00107
:1016B0001124E45DFE4F20E030E070E04081CB017A
:1016C000022E02C0969587950A94E2F78170819563
:1016D00084278523842781932F5F3F4F2530310551
:1016E00069F708952FE0929F800D1124682F669569
:1016F00066956695982F977085E0689FB0011124D4
:1017000040E050E080E0FB01E40FF51FE45DFE4F98
:10171000208130E0092E02C0369527950A94E2F721
:1017200021703327042E01C0220F0A94EAF7822B7E
:101730004F5F5F4F4530510531F70895BF92CF920B
:10174000DF92EF92FF920F931F93CF93DF938C0161
:10175000C0906801D0906901E0906A01F0906B013F
:1017600080916C0190916D01A0916E01B0916F011B
:10177000C82AD92AEA2AFB2ACFE1D0E0D701C6013C
:101780000C2E04C0B695A795979587950A94D2F725
:1017900080FD04C0219790F7B12C07C0BC2EB80182
:1017A0008C2F0E94D9120197A9F38B2DDF91CF9135
:1017B0001F910F91FF90EF90DF90CF90BF90089511
:1017C000CF93DF93EC010E949E0BBE010E94D912C1
:1017D000DF91CF9108951F93CF93DF93EB01909109
:1017E0002B01992321F0CB010E94E00B13C0882329
:1017F00049F0CB010E949E0B182F682FCE010E944A
:10180000470B04C0CB010E94720B182FBE01812F21
:101810000E94D912DF91CF911F9108951F93CF930A
:10182000DF93C091700116E080917101C81799F0A3
:10183000D0E01C9FF0011D9FF00D1124EE58FE4FCB
:101840004081518162817381848195810E94270A40
:101850002196C770E9CFDF91CF911F9108954091F4
:10186000A2015091A3016091A4017091A501809102
:10187000A6019091A7010C94270AEF92FF920F9373
:101880001F93CF93DF938091A70182958F7009F00A
:1018900065C08091A401882309F460C08091700123
:1018A000F09071011091A2010091A3016091A50136
:1018B0007091A60191E01F3F09F090E0C091620095
:1018C000D0916300292F96E0E92E8F1509F446C0C8
:1018D0006115710521F00F3F21F030E003C031E0C8
:1018E00001C0322F90E030FD36C0E89EF001E99E45
:1018F000F00D1124DF01AE58BE4F11963C911197A7
:10190000301329C03C91311326C012963C91129796
:10191000311121C013964D915C911497461B570BC2
:101920004C175D07C0F48091A7018F708061809390
:10193000A701E958FE4F80818F708061808382EA21
:1019400091E00E94A909DF91CF911F910F91FF9023
:10195000EF900C940E0C01968770B7CFDF91CF916A
:101960001F910F91FF90EF9008959F92AF92BF92B9
:10197000CF92DF92EF92FF920F931F93CF93DF935B
:10198000CDB7DEB761970FB6F894DEBF0FBECDBFFF
:101990008C0185E0F801DE011D9601900D928A957B
:1019A000E1F7D8011296EC909091A201E091A30189
:1019B0002091A5013091A6012115310531F0EF3FAD
:1019C00031F481E09F3F19F403C081E001C080E061
:1019D000B82FB1709B2E80FD47C1D8014C91119654
:1019E0005C9111971396AD90BC90149782EAC82E23
:1019F00081E0D82EF090A401B501621B730B2091F9
:101A0000620030916300FF2009F4D9C08091A701E2
:101A10006217730708F095C0282F207F09F052C085
:101A20005E1313C0491311C0FE2CE1100EC08F705D
:101A300080618093A7010E942F0CC6010E94A90912
:101A40008091A701F80185834DC1AB2831F05F3F3C
:101A500031F481E04F3F19F403C081E001C080E020
:101A600080FD03C081E08E2502C080E090E0F82F69
:101A7000F170FF2E80FF1CC08091700120917101D8
:101A800036E0821709F40BC190E0389FF001399FCE
:101A9000F00D1124EE58FE4F6181561306C060818F
:101AA000461303C06281E61203C001968770E9CF36
:101AB000FE2CEE2009F416C18091A701816080936D
:101AC000A70154C05E1306C0491304C0E11002C050
:101AD000F80199C0C8010E94100A882361F1EE2024
:101AE00051F12091A701822F82958F7090E002978B
:101AF00074F08091A2019091A30198878F83198639
:101B0000BB86AA862C87CE0107960E94A90986E08B
:101B1000F801A2EAB1E001900D928A95E1F70E94E6
:101B20003D0C0E942F0C0AC05E1711F1C8010E94E3
:101B3000100A81112CC0C8010E94A909FF24F39446
:101B4000D1C0282F207F81F77A2DB98AA88A6E2DDF
:101B500089890E94180A82EA91E00E94A90986E018
:101B6000D6011D928A95E9F70E942F0CF12CBAC07C
:101B70004913DCCFE110DACFF8018583C8010E9458
:101B8000A90986E0D6011D928A95E9F7ABC0EE203F
:101B900091F22091A701822F82958F7090E0029799
:101BA0000CF4B5CF8091A2019091A3019A8389830F
:101BB0001B82BD82AC822E83CE010196A6CF621716
:101BC000730708F044C0FE2CEE2009F4B4CF5E1376
:101BD00030C049132EC02091A70120FD21C0822FC3
:101BE00082958F70482F50E041155105C9F0F801DA
:101BF00025834F30510541F08F5F982F9295907F4C
:101C0000822F8F70892B8583C8010E94A90986E0E5
:101C1000F801A2EAB1E001900D928A95E1F73CC08B
:101C200086E0F801A2EAB1E001900D928A95E1F711
:101C300059C0C8010E94100A811169CF8091A70183
:101C400081608093A701C8010E94A9094BC07A2D29
:101C5000B98AA88A6E2D89890E94180A86E0D60161
:101C60001D928A95E9F718C0EE2009F464CFC801E7
:101C70000E94100AF82E882309F45DCF86E0F8014F
:101C8000A2EAB1E001900D928A95E1F782EA91E033
:101C90000E94B8060E943D0C0E942F0C23C04D8765
:101CA0005E878D859E850E94E00B292F22952F70DF
:101CB000223028F49F7039F0811105C00BC0243008
:101CC00028F49F7049F4805E883020F0C8010E949B
:101CD000A9099F2CF92C06C0D80115969C91907FDC
:101CE00091F7F8CF8F2D61960FB6F894DEBF0FBE37
:101CF000CDBFDF91CF911F910F91FF90EF90DF90BB
:101D0000CF90BF90AF909F9008951F93CF93DF9394
:101D1000CDB7DEB72C970FB6F894DEBF0FBECDBFA0
:101D20004F83588769877A878B879C87CE01079670
:101D30000E94B50C8823D1F09F8188852A853B8538
:101D4000232B31F08F3F31F481E09F3F19F403C022
:101D500081E001C080E080FD47C04F8158856985E2
:101D60007A858B859C850E94270A3EC086E0FE010D
:101D70003796DE01119601900D928A95E1F7FF8169
:101D8000E8856A857B856115710531F0EF3F31F497
:101D900081E0FF3F19F403C081E001C080E080FDD5
:101DA00023C02091710130E0C90101968770992705
:101DB0004091700150E084179507F1F1F983EA83AF
:101DC0007D836C8396E0929FD001939FB00D112488
:101DD000AE58BE4FFE01319601900D929A95E1F7F3
:101DE000809371010E940E0C16E080917001909119
:101DF0007101891771F1189FC00111248E589E4FEF
:101E00000E94B50C882329F1E09170011E9FF0011A
:101E10001124EE58FE4F408151816281738184818B
:101E200095810E94270A8091700190E00196877049
:101E3000992780937001D9CF0E94F1091092710106
:101E400010927001E2EAF1E086E0DF011D928A95CE
:101E5000E9F72C960FB6F894DEBF0FBECDBFDF9129
:101E6000CF911F9108958091B001859585958595B5
:101E700008958091B001877008959091B001977096
:101E800081E009F480E008958091BB01089590916C
:101E9000BB01892B8093BB01089580959091BB0174
:101EA00089238093BB0108951092BB0108959091FE
:101EB000BA01892B8093BA01089580959091BA0157
:101EC00089238093BA0108951092BA0108958091F0
:101ED000B101089508950C946A0F0C946B0F9091C2
:101EE000870292FD08C09091B101981721F080936C
:101EF000B1010C946D0F08958091B101882329F0F0
:101F00001092B10180E00C946D0F0895CF93DF9390
:101F1000E0916400F09165008091BB018083E091C5
:101F20006400F091650090818091BA01892B8083D3
:101F30008091B101882381F0E0916400F091650007
:101F40009081892B808380916400909165000E942C
:101F5000712081110E947C0FC0916400D0916500B6
:101F600048E050E068EA71E0CE010E94EB24892B42
:101F700069F088E0FE01A8EAB1E001900D928A952F
:101F8000E1F7CE01DF91CF910C943A20DF91CF9110
:101F900008950C946A0F9091870292FD10C098E00A
:101FA000899F90011124262B2093B0010E94A90A39
:101FB0008091B0018595859585950C94C90F0C94F9
:101FC000A90A1092B00180E00C94C90F2091B001D1
:101FD000809582238093B001982F977099F430E018
:101FE000482F082E000C550B2417350759F09091F7
:101FF000870292FD07C08595859585950E94CA0A3E
:102000000C94E10F08959091870292FB222720F90A
:10201000281769F080FB92F99093870280918602DD
:10202000909187020E94511082E00C94E60F08956F
:102030008091870282FB882780F991E089270C94A0
:10204000031081E00C94031080E00C9403106FEFF8
:102050007FEF80E090E00C94292580E090E00E94E2
:10206000062521E0893E9E4F09F020E0822F089549
:1020700082E090E00C94F82483E090E00C94F82443
:10208000CF9384E090E00E94F824C82F82E290E091
:102090000E94F8242C2F30E0A901582BCA01CF91BF
:1020A0000895CF93C92F682F84E090E00E940C25FB
:1020B0006C2F82E290E0CF910C940C25AB01BC0117
:1020C0008FE090E00C941D25AB01BC0183E190E012
:1020D0000C941D2560E070E0CB010C94641060E06E
:1020E00070E0CB010E945E100C946A1069EE7EEFE6
:1020F00080E090E00E94292560E082E090E00E946C
:102100000C2560E083E090E00E940C2510926C01A9
:1021100010926D0110926E0110926F0160E084E0E8
:1021200090E00E940C2560E082E290E00E940C2585
:1021300060E085E090E00E940C2560E086E090E0A1
:102140000E940C256FEF87E090E00E940C2540E094
:1021500050E0BA0188E090E00E941D2560E08DE02B
:1021600090E00E940C2540E050E0BA0188E190E048
:102170000E941D2560E087E190E00E940C2540E070
:1021800050E0BA018CE190E00E941D2560E070E013
:1021900080E290E00E94292540E050E0BA0188E109
:1021A00090E00E941D250C946F100C947610682FFF
:1021B0008EE090E00C940C250E94FC206093CC01F2
:1021C0007093CD018093CE019093CF016093C801AD
:1021D0007093C9018093CA019093CB01089584B78D
:1021E000806884BF84B7806884BF089581E00895C3
:1021F0000C94F61008950C94FA100C94FA100C94A8
:10220000FD100C94FA100C9401110C94FA100E9419
:10221000EF1085EB93E10E9424200E9405110C949D
:1022200003110E94FB100C94FA100E94D2130C941C
:1022300052060E94E9200E9456040E9415110E9435
:10224000C5190C94FF105F926F927F928F929F92AC
:10225000AF92BF92CF92DF92EF92FF920F931F93B4
:10226000CF93DF93CDB7DEB72A970FB6F894DEBFD2
:102270000FBECDBF0E947B04C82E81110E94DC10CE
:102280003CEB832E31E0932E00E010E0502E802FA7
:102290000E9414055C01F401619071904F01682661
:1022A000792661147104B1F40F5F1F4F06301105D8
:1022B00069F78FEF89838A831B820E94F0208160F7
:1022C000782F9D838C8349815A816B818D810E94F7
:1022D0006E063AC08091D00181FD0E941D05D12C6F
:1022E000EE24E394F12CC3018E219F21892B29F147
:1022F0000E94F8108823A9F0DE825F82AE20BF2002
:1023000081E0AB2809F480E088870E94F02081609A
:10231000782F9A8789874E815F8168858A850E9498
:102320006E06000F111FF801E454FE4F8081918169
:10233000E826F926F182E08207C0D394EE0CFF1C58
:10234000FFE0DF12D0CFB0CF81E0C11001C080E04C
:102350002A960FB6F894DEBF0FBECDBFDF91CF91A6
:102360001F910F91FF90EF90DF90CF90BF90AF90B3
:102370009F908F907F906F905F9008950E9423119F
:102380000E94091A0C946306CF93DF930E94DE1219
:10239000EC01811522E59207E8F5811531E59307F7
:1023A00008F0B6C0883E910528F5803E910508F0FA
:1023B000E9C0883A910570F4853A910508F07AC031
:1023C0008130910509F473C008F4D9C0049708F06E
:1023D000D9C0D5C08F3B910508F0D1C0C85AD0E014
:1023E000CC0FDD1FC854DF4F0990D881C02DCE011E
:1023F0009464C9C0811540E5940708F069C081154F
:1024000050E4950708F060C09A9581159F4108F443
:10241000B9C0B5C0811536E5930728F5811545E5A6
:10242000940708F092C0811554E5950708F087C01D
:10243000AC0143705527282F26952695C115D34505
:1024400008F06CC081E090E002C0880F991F4A95A7
:10245000E2F740E2249F90011124EC01C22BD32B20
:10246000CE019C6890C081152AE5920780F4811501
:1024700039E5930708F072C0811548E5940708F420
:102480007EC0D82FCC27CE01806F906A7CC090563A
:102490008115904208F073C08D2F8F710E947213C6
:1024A000DD27D0628F71AE01582BCA016CC081E06C
:1024B00090E069C0C55AD0E0CA51DF4F8881C82F6B
:1024C000D0E0CE0190645FC0DF70CE01906A5BC047
:1024D00074E0969587957A95E1F7282F23703C2F25
:1024E000337081E090E002C0880F991F3A95E2F7BF
:1024F0009C68AC01522B9A019C2F9F7096959695E3
:1025000050E2959FE0011124C9018C2B9D2B3BC00B
:10251000D82FCC27CE01816F906A35C081E090E042
:1025200002C0880F991F4A95E2F750E2259F90015B
:102530001124EC01C22BD32BCE019A6824C0D82FD2
:10254000CC27CE01846F906A1EC00E9472138F71D7
:1025500090E0D82FCC27CE01906215C08F700E94DA
:10256000721394E0D695C7959A95E1F7CF70D0E0B5
:10257000DC2FCC27D0699E01282BC90104C080E044
:1025800090E001C0CE01DF91CF9108952AE5829FAE
:10259000C0011124FC012FE0729FE00DF11D1124F8
:1025A000E60FF11DEE0FFF1FE459FF4F8591949147
:1025B00008950E94C6120E94C411089582389105A0
:1025C00069F1B0F48133910509F46DC048F48932A2
:1025D000910509F463C08A32910509F469C0089530
:1025E0008533910509F455C089339105B9F00895F3
:1025F000833E910569F138F4803E9105B1F0823E49
:10260000910509F10895863E9105A9F1873E91054E
:10261000B9F1843E910509F064C023C0209186027F
:1026200020FD4FC021FD4DC008958091860280FDA0
:1026300044C08091870280FF44C08091860284FD5F
:1026400042C083EE4DC08091860282FF38C0F5CF34
:102650008091860282FD33C08091870280FD31C067
:10266000ECCF8091870281FF32C08091860284FD89
:102670002AC087EE35C08091860283FF26C0F5CF41
:102680008091860283FD21C08091870281FD1FC059
:10269000ECCF8091860285FD1CC01DC08091860212
:1026A00085FD19C016C08091860286FD16C017C030
:1026B0008091860286FD13C010C089E311C082EEAE
:1026C0000FC080EE0DC080E00BC086EE09C084EE26
:1026D00007C089E205C085E303C08AE201C081E347
:1026E00090E008959091860292FF0DC0282F2871E6
:1026F000283019F4877F846006C0282F2471243085
:1027000011F48B7F886093FF0DC0282F287128312A
:1027100019F4877E846106C0282F2471243111F4B6
:102720008B7E88612091870220FF0DC0382F387181
:10273000383019F4877F816006C0382F317131300D
:1027400011F48E7F886021FF0DC0282F2871283159
:1027500019F4877E816106C0282F2171213111F47F
:102760008E7E886194FD877E089580E008950C94A4
:1027700027100E947B042FE389E191E021508040E3
:102780009040E1F700C000000E947B0480E00E94BE
:10279000140580FF04C00E94B7130C943D210895D6
:1027A0000C94B9130E942D10811102C00E94D51003
:1027B0000E9438108093D0010E94401090938702AD
:1027C000809386020E94D0130E943C10682F70E014
:1027D00080E090E00E94490A60916801709169016F
:1027E00080916A0190916B010C94810A0895FF9287
:1027F0000F931F93CF93DF93F82E092F162FD72F08
:10280000C42F222349F081E08093D3010E94F0205D
:102810009093D2018093D1018091D3018823D9F084
:102820008091D1019091D2010E940821059798F0E2
:10283000EF2DF02FA12FBD2F80E090E04C2F50E026
:102840008417950734F4219131912D933D9301968E
:10285000F7CF1092D301DF91CF911F910F91FF908D
:1028600008950E9452210E9419110C9463210E9424
:10287000DE200E944B210E9407110E9431140E9409
:1028800071210E941111FBCFEF92FF920F931F93C2
:10289000CF93DF938B01682F11110AC0442329F0D5
:1028A000E82FF0E0E156FC4F6491762F862F75C03B
:1028B000212F30E0E82FF0E0442321F0E156FC4FD7
:1028C000E491F0E046E0049FC0011124CFEFD0E096
:1028D000BE010E9451244BEA4603C001479F900D60
:1028E0001124800F911D800F911D982F990F890F32
:1028F000AE01421B530B4E9FD0014F9FB00D5E9F08
:10290000B00D11249B2F189FA0011124452F55278E
:102910008E01041B150B0E9FA0010F9F500D1E9FD3
:10292000500D11247E01E81AF108E29E8001E39E19
:10293000100DF29E100D1124212F3327C21BD30B33
:10294000CE9F9001CF9F300DDE9F300D112462305D
:102950007105A9F048F46115710569F061307105E0
:10296000C9F48B2F752F0DC06430710581F058F0BC
:102970006630710579F47E2F8B2F932F0DC0832F36
:102980007B2F9E2F09C08E2F7B2F952F05C08E2F5A
:10299000732F02C07E2F852F692FDF91CF911F915A
:1029A0000F91FF90EF90089541E00E944414089524
:1029B00008950E94D4140895CF93DF93762FE901F0
:1029C000682F842F0E94D914798368838A83DF91CA
:1029D000CF9108954B3F08F04AEF0C94DC1480919E
:1029E0008802282F269530E02115310519F48170D1
:1029F000826005C02532310524F08170886480939F
:102A0000880280918B028B3F18F08AEF80938B02B3
:102A1000089588E090E00C940025CF92DF92EF9229
:102A2000FF926B017C010E94EF14B701A60188E0C0
:102A300090E0FF90EF90DF90CF900C941D25E8E898
:102A4000F2E083E0808311828FEF82838AEF8383B9
:102A5000148260817181828193810C940D15809123
:102A6000880280FF02C08695089580E008959091C5
:102A70008C02933018F49F5F90938C02882351F05E
:102A8000609188027091890280918A0290918B02F4
:102A90000C940D15089581E00C94371590918C02DB
:102AA000992319F0915090938C02882351F06091F2
:102AB00088027091890280918A0290918B020C9415
:102AC0000D15089581E00C944E1570E00C94861B52
:102AD00060916A008091880280FF0AC0809169003D
:102AE00023E0829FC001112483579D4F0C946515EC
:102AF00080916B0090916C00891780F7E82FF0E0CF
:102B00009F01220F331FE20FF31FE357FD4F118286
:102B1000108212828F5FF0CF9091880290FF16C0D2
:102B200090916B0020916C00921770F4E92FF0E007
:102B3000DF01AA0FBB1FEA0FFB1FE357FD4F818385
:102B4000608342839F5FF0CF0C9468150895CF9304
:102B5000DF9300D01F92CDB7DEB79091880290FF2F
:102B60000AC09E012F5F3F4F0E94EA144B8169818A
:102B70008A810E948C150F900F900F90DF91CF915A
:102B80000895CF93DF93EC01EC81F0E0E656FD4F22
:102B90004491E8E8F2E0628181810E94A7158C816E
:102BA0008F5F8C83DF91CF910895CF93DF93EC01FA
:102BB000E8E8F2E0438162818C810E94A7158C8154
:102BC0008F5F8C83DF91CF9108950F931F93CF93E5
:102BD000DF9300D01F92CDB7DEB78C018091D40176
:102BE00081110AC09E012F5F3F4F4AEF6FEF0E9495
:102BF000EA148A818093D401F8018481813051F0F4
:102C000028F0823061F44091D4010AC08091D4014F
:102C100040E007C06091D40140E080E003C040E0A4
:102C200080E060E00E948C15F801848190E00196BC
:102C300063E070E00E94652484830F900F900F90F2
:102C4000DF91CF911F910F910895AF92BF92CF92D4
:102C5000DF92EF92FF920F931F93CF93DF9300D0F9
:102C60001F92CDB7DEB7182FF62E042FE22E9091CB
:102C7000880290FF6DC0E92FE695AE2FB0E0A75116
:102C8000BF4F8C918093E0019E7F923061F49E0152
:102C90002F5F3F4F812F0E94EA144B8169818A8107
:102CA0000E948C1543C0823019F400918B023EC003
:102CB000863019F41091890239C08930D9F38931ED
:102CC000A9F5E9518E2F8170D82EE695F0E0E656F1
:102CD000FC4FA590B490C12CBB2460916D00C6162A
:102CE00018F52C2D30E0A29EC001A39E900DB29E3F
:102CF000900D112470E00E945124812FD11002C048
:102D0000860F01C0861B90916B00290F311DA90110
:102D1000440F551F240F351F23573D4F402F6F2D54
:102D20000E94EA14C394D9CF0E94681510938902B7
:102D3000F0928A0200938B02EE2051F0609188029B
:102D40007091890280918A0290918B020E940D15E8
:102D50000F900F900F90DF91CF911F910F91FF90E7
:102D6000EF90DF90CF90BF90AF900895E8E8F2E049
:102D70009181282F4381628188E0890F0C94251668
:102D800081E00C94B616E8E8F2E09181282F4381A7
:102D9000628188EF890F0C94251681E00C94C3168C
:102DA000E8E8F2E0628128E0620F08F46FEF282F74
:102DB000438181810C94251681E00C94D016E8E8BB
:102DC000F2E0628128E0621B08F460E0282F438172
:102DD00081810C94251681E00C94DF16E8E8F2E07E
:102DE000438128E0420F08F44FEF282F6281818150
:102DF0000C94251681E00C94EE16E8E8F2E043818D
:102E000028E0421B08F440E0282F628181810C9465
:102E1000251681E00C94FD1620E00C942516FF92F7
:102E20000F931F93CF93DF93EC01F12C0FEF10E082
:102E300060916D00F616F0F480916B002F2D30E05C
:102E4000280F311DC901880F991F280F391F2357DB
:102E50003D4F70E0C8010E946524962F8C814091FF
:102E60008B0260918A02F99E800D11240E94EA145F
:102E7000F394DECF0E9468159A818C8190FF02C086
:102E80008F5F01C081508C83DF91CF911F910F9193
:102E9000FF900895AF92BF92CF92DF92EF92FF9290
:102EA0000F931F93CF93DF93FC01828180FF02C0B9
:102EB0000FEF01C001E010E04CE0A42E80916D0006
:102EC000181708F043C080916B00C12ED12CE60189
:102ED000C80FD11DCE01880F991FC80FD91FC35726
:102EE000DD4F198218821A8234E0E32EF12CB12CC6
:102EF0008091D6018B0D8D302CF06A2D0E944324D9
:102F0000892F05C087FF03C090916D00890F082E9F
:102F1000000C990BC816D90691F480918B028E9DF6
:102F2000A0018F9D500D11245595479555954795B6
:102F30009E0160918A02809189020E94EA14B00E7B
:102F4000F1E0EF1AF108A1F61F5FB8CF0E946815F3
:102F50008091D601013031F4811102C080916D0061
:102F6000815007C090E0019660916D0070E00E9472
:102F700065248093D601DF91CF911F910F91FF902F
:102F8000EF90DF90CF90BF90AF900895CF93809156
:102F90006B0090916C00891770F4E82FF0E09F01AE
:102FA000220F331FE20FF31FE357FD4F11821082F0
:102FB00012828F5FF0CFC0E060916D00C617C0F540
:102FC000EC2FF0E070E0CF010E94652420916B00AF
:102FD000820F2091D501022E000C330B90E0E217F6
:102FE000F307CCF020916800022E000C330B2E1753
:102FF0003F078CF09C01220F331F820F931F9C010F
:1030000023573D4F40918B0260918A028091890243
:103010000E94EA140BC0FC01EE0FFF1F8E0F9F1FD2
:10302000FC01E357FD4F118210821282CF5FC4CFA3
:103030000E946815209167008091D501820F8093CE
:10304000D50190916800920F9093680019165CF476
:10305000082E000C990B40916D0050E04150510931
:10306000841795071CF0219520936700CF91089550
:103070008F929F92AF92BF92CF92DF92EF92FF9288
:103080000F931F93CF93DF938C01FC014481C42FD6
:10309000D0E09E01DE010E94A9249B01AC010E94A8
:1030A000BF246B017C01E0E2F0E0EC1BFD0BA5E529
:1030B000B0E09B01AC010E94BF244B015C019F0169
:1030C000DF010E94A1249B01AC010E94CA249B0144
:1030D000AC012C0D3D1D4E1D5F1DC501B4010E94AC
:1030E0007924C22FD22F2A3228F4F3E02F9F9001A7
:1030F00011240DC025E530E02C1B3109C901880FD2
:10310000991F280F391F37FF02C02F5F3F4F35959A
:103110002795C22FC095F12C85E5E82EED1A8091F8
:103120006D00F816C8F4F1FC02C08E2D01C08D2F81
:1031300090916B002F2D30E0290F311DA901440F14
:10314000551F240F351F23573D4F4C2F60918A0286
:103150000E94EA14F394E3CF0E946815F801848179
:10316000811102C091E003C0803219F49FEF909367
:10317000660090916600890FF8018483DF91CF91FA
:103180001F910F91FF90EF90DF90CF90BF90AF9085
:103190009F908F9008950F931F93CF93DF93EC012F
:1031A00000E010E080916D00282F30E00217130737
:1031B00024F590916B009801290F311DA901440F4E
:1031C000551F240F351F23573D4F869590E04C81A6
:1031D000081719071CF4442331F002C0411103C041
:1031E00040918B0201C040E060918A028091890287
:1031F0000E94EA140F5F1F4FD5CF0E9468158C8183
:1032000090E00196817099278C83DF91CF911F9177
:103210000F910895E8E8F2E080818E7F80836081DD
:103220007181828193810E940D151092E1012FEB33
:1032300084ED91E0215080409040E1F700C0000013
:103240000C946815E8E8F2E080818E7F808310920C
:10325000E1012FEB84ED91E0215080409040E1F7B7
:1032600000C000000C9468151092E1018091DE010D
:1032700081110AC081E08093DE0180918802817013
:103280008093DD010C94221908956091880266955F
:1032900070E04BE050E08EE690E00E94DE24892B47
:1032A00019F481E08093E1010E94F0209093D8010D
:1032B0008093D70108959091880290FF35C0917056
:1032C000811102C0926006C0853210F0986402C07D
:1032D000880F982B90938802662351F060918802A2
:1032E0007091890280918A0290918B020E940D1543
:1032F00060918802669570E04BE050E08EE690E0C9
:103300000E94DE24892B19F01092E10102C00E9474
:10331000451981E08093DA0140918B0260918A0225
:10332000809189020C940C170895682F909188025F
:10333000969581E0890F853208F081E00C945B1945
:1033400081E00C949519682F9091880296958FEFE3
:10335000890F09F484E20C945B1981E00C94A319A1
:1033600061E00C945B19E8E8F2E080818160808381
:1033700086950C94B0198091880280FD0C940A19EE
:103380000C94B31960E00C945B198091DF018111FA
:103390002EC00E942D10811104C00E94D5100E94E1
:1033A0001F150E940915609388027093890280930B
:1033B0008A0290938B026E7F61F40E941F150E9417
:1033C0000915609388027093890280938A02909312
:1033D0008B020E94EF141092E1018091880280FF1D
:1033E00003C086950E94C21981E08093DF01089591
:1033F000E8E8F2E080818160808386950C94C219B0
:103400001092DE018091DD0181110E94F8190C9467
:1034100045190F931F93CF93DF938091E101882388
:1034200009F485C08091E001E0918802E695E81BEF
:10343000E093D901823049F4F0E0EA56FD4FE4917F
:10344000CE2FD0E001EC15E149C0863049F4F0E020
:10345000ED56FD4FE491CE2FD0E005ED15E13EC0D5
:10346000893051F4E695F0E0E057FD4FE491CE2F1E
:10347000D0E00FE017E132C08F3051F4E695F0E074
:10348000E357FD4FE491CE2FD0E00AE417E126C0C8
:10349000853149F4F0E0E657FD4FE491CE2FD0E0BE
:1034A00006EC17E11BC0883181F0833239F4E8E87B
:1034B000F2E0C591D49105EE15E110C0843251F4CB
:1034C000C4EFD1E00BEC18E109C0C8E2D0E008E39A
:1034D00018E104C0C0EDD7E008ED14E18091DA01F5
:1034E000882361F01092DA010E94F0209093D801B5
:1034F0008093D7011092DC011092DB010E94F02032
:10350000E091D701F091D8018E1B9F0B8F3F9F4711
:1035100070F4EC0FFD1FF093D801E093D70187ED15
:1035200091E0F801DF91CF911F910F910994DF9104
:10353000CF911F910F910895882311F0FA0101C0D6
:10354000FB010994CF93DF93C82FD62F0E942F152C
:103550008C1740F00E942F158D1720F4DF91CF912A
:103560000C94A0198C2FDF91CF910C94B0191F935C
:10357000CF93DF93FB0112811111C3C0EC010E94B4
:10358000440F8272CD3CFCE5DF0709F49AC0A8F530
:10359000C73CECE5DE0709F476C0A8F4C43C9CE522
:1035A000D90709F45FC028F4C33CDC4509F457C0CF
:1035B00054C0C53C9CE5D90709F459C0C63CDC455C
:1035C00009F45CC04AC0CA3CFCE5DF0709F46AC0E4
:1035D00050F4C83CECE5DE0709F45AC0C93CDC45B0
:1035E00009F45BC03AC0CB3C9CE5D90709F45FC045
:1035F000CC3CDC4509F460C030C0C23DFCE5DF07CF
:1036000009F46FC088F4CF3C9CE5D90709F460C089
:1036100008F45CC0C03DFCE5DF0709F45CC0C13DB7
:10362000DC4509F45BC019C0C53D9CE5D90709F428
:1036300060C050F4C33DFCE5DF0709F455C0C43D4C
:10364000DC4509F454C009C0C63D9CE5D90709F41E
:1036500055C0CE35DD4509F454C011E052C00E947A
:10366000BB194FC04DEA59E160EA79E104C040EA74
:1036700059E16DEA79E10E949C1A43C04DEC56E194
:1036800060EC76E1F8CF40EC56E16DEC76E1F3CFFB
:103690004BEE56E16CED76E1EECF4CED56E16BEE84
:1036A00076E1E9CF49E057E16AEF76E1E4CF4AEF0E
:1036B00056E169E077E1DFCF42E655E16BE475E181
:1036C000DACF4BE455E162E675E1D5CF81E017C072
:1036D00065E082E010C068E086E00DC06EE089E041
:1036E0000AC064E18FE007C067E185E104C088E1BA
:1036F00006C062E289E10E94A21A03C083E20E942E
:10370000B019812FDF91CF911F9108950F931F93CF
:10371000CF93DF938C01EB018091E201811105C011
:103720000E94CA1E81E08093E201AE01440F551F42
:103730004C0F5D1F24E630E0B80180EBDF91CF91A4
:103740001F910F910C94C11FCF93DF93EC01FB01EC
:103750008281882309F43CC1C430FDE5DF0760F4B1
:10376000CB3F9CE5D90788F49E0122503C4524318B
:10377000310508F02EC109C0C236EDE5DE0729F09B
:10378000C63AFDE5DF0709F024C10E94401090937E
:10379000870280938602C1318CE5D80709F4C6C040
:1037A00008F042C0C930ECE5DE0709F49BC000F523
:1037B000C5308CE5D80709F485C078F4C330ECE552
:1037C000DE0709F478C008F07AC0C230DC4509F0A1
:1037D000F5C0809186028160EFC0C7309CE5D907B3
:1037E00009F478C008F07AC0809186028061E4C054
:1037F000CD30FCE5DF0709F487C058F4CB309CE5F9
:10380000D90709F479C008F07BC0809186028860EE
:103810006FC0CF30FCE5DF0709F480C008F082C03C
:1038200080918602877FC8C0CE3F9CE5D90709F406
:1038300071C000F5C531FCE5DF0709F485C068F407
:10384000C3319CE5D90709F475C008F095C00E9402
:10385000F109809186028F77AFC0CC3FFCE5DF078E
:10386000A9F108F054C0CB3FDC4509F0A7C0809116
:10387000870240C0C230EDE5DE0709F489C058F484
:10388000C1158DE5D80709F45AC008F069C08091C8
:10389000870282602FC0C236EDE5DE0709F47CC0E6
:1038A000C63AFDE5DF0709F481C0C330DD4509F004
:1038B00085C080E06EC08091860282607DC080916C
:1038C000860216C080918602886076C08091870249
:1038D00082604FC08091860280626EC080918602B5
:1038E00080646AC00E94F10980918602806864C089
:1038F000846062C081603DC0809186028E7F5CC022
:10390000809186028D7F58C08091860216C080917A
:10391000870218C0809187028D7F2BC0809186021C
:103920008F7E4AC0809186028F7D46C0809186023C
:103930008F7B42C080918602877F8B7F3DC08091C4
:1039400087028D7F8E7F15C08091860282FB2227A1
:1039500020F991E0922790FB82F990FB83F92CC02B
:1039600080918702982F909591708E7F892B90FB84
:1039700081F98093870222C00E94F109809186021A
:1039800087FB222720F991E0922790FB87F914C04A
:1039900081E00E94D71012C08091860284FB22270A
:1039A00020F991E0922790FB84F906C0809186026D
:1039B000982F909590FB80F98093860280918602E3
:1039C000909187020E9451100E94F10980E001C08D
:1039D00081E0DF91CF9108950F931F9341E050E074
:1039E00060E070E08A019B0104C0000F111F221FDC
:1039F000331F8A95D2F7C901B8010E94490A1F9165
:103A00000F910C94F1098B3109F468C058F58B3093
:103A100009F486C078F4863009F445C020F4853076
:103A200009F44BC07FC0873009F44AC0883009F4DC
:103A300077C078C0803109F464C068F48E3009F032
:103A400071C08091D00182FB222720F991E092275A
:103A500090FB82F94CC0863109F462C0893109F4C7
:103A60005FC060C08A32E1F060F4873209F455C06B
:103A700028F48E3108F456C08D5150C08932E9F0D7
:103A800051C0833450F48A3308F045C0853309F4BB
:103A900044C0883309F444C045C08334F1F142C0C6
:103AA0000E94D5103DC08091D001817F8E7F809390
:103AB000D00181E08093E30108950E94D70530C0D2
:103AC0008091D001982F9095917090FB80F9809310
:103AD000D001911125C0897F877F10C08091D001CE
:103AE00081FB222720F991E0922790FB81F98093B6
:103AF000D0019923A9F08091D00181608093D001F9
:103B00000FC08091D00183FB222720F991E09227FA
:103B100090FB83F9ECCF895301C080E00E94EC1C3C
:103B200081E0089580E0089580E008950C94941D4C
:103B3000CF93C82F8091E301882319F0813031F0B1
:103B40002BC00E94440F823249F504C00E94440FEA
:103B5000823261F48C2F0E94961D811104C08C2F3B
:103B60000E94031D17C081E090E014C08C2F0E94BA
:103B7000941D81110EC0C43149F018F4CB3049F0C6
:103B80000FC0C93219F0C83321F00AC01092E30106
:103B900007C081E0817006C01092E30180E002C09E
:103BA00080E0F8CFCF910895CF93DF9386319C4585
:103BB00041F5EB010E94440F982F8A812091640007
:103BC00030916500882379F09A7A81E009F480E0E9
:103BD0008093E401911102C069E201C065E3C9016B
:103BE0000E94B3200AC08091E401811102C069E201
:103BF00001C065E3C9010E94B5200E94860F80E0E4
:103C000001C081E0DF91CF9108950F931F93CF936F
:103C1000DF93C42FD22FFC0182818823C9F0409307
:103C2000E7010E94F0209093E6018093E50180E295
:103C30008C0F883008F057C0C77081E001C0880F32
:103C4000CA95EAF7DF91CF911F910F910C945D0710
:103C50008091E701481330C08091E5019091E60121
:103C60000E940821883C910538F510E21D0FCD1700
:103C7000B9F080E28C0F883040F4C77081E001C059
:103C8000880FCA95EAF70E946407183028F581E08A
:103C90009D2F977001C0880F9A95EAF70E945D07E3
:103CA000802F0E9454071830F0F4D77081E001C0D3
:103CB000880FDA95EAF70AC080E28C0F883098F412
:103CC000C77081E001C0880FCA95EAF7DF91CF91F4
:103CD0001F910F910C946407802FDF91CF911F915A
:103CE0000F910C945407DF91CF911F910F9108957C
:103CF0000F939C01CB01243F4CE5340731F188F44C
:103D0000293DFCE53F07D9F02A3D4CE5340779F120
:103D1000283D3C45A9F506E221EE41EE68ED7CE543
:103D20002BC0263FFCE53F07E1F0A8F0273F3C45CC
:103D300039F507E225EE46EE67EF7CE51DC007E2A8
:103D400025EE45EE69ED7CE517C006E221EE40EE7A
:103D500064EF7CE511C007E225EE44EE65EF7CE5FB
:103D60000BC006E221EE42EE66EF7CE505C008E2FC
:103D700021E045EE6AED7CE50E94051E80E008C06A
:103D8000FC018281882319F01092E70101C081E0D3
:103D90000F91089511B887E080B985B3836085BB22
:103DA00086B7846086BF86B7816086BF86B7806429
:103DB00086BF08959F92AF92BF92CF92DF92EF920B
:103DC000FF920F931F93CF93DF93B82EEB010E94C6
:103DD000F0206C01C431D10558F0CF3F8FEFD807E8
:103DE00059F0CE0164E170E00E9451247B0107C0CC
:103DF000EE24E394F12C03C025E0E22EF12C84E8BC
:103E0000A82E94EA992E16BE96BE0E94F0208C0130
:103E100006B607FC08C00E94F020801B910B8E158F
:103E20009F05B0F324C081B1887F883039F081B11B
:103E3000887F803119F00FEF1FEF1BC0B3B8A6BE0B
:103E40000E94F0208C0106B607FC08C00E94F020FA
:103E5000801B910B8E159F05B0F309C081B1887F3F
:103E6000883111F0803439F700E010E00DC00EEF1A
:103E70001FEFCF3F8FEFD80731F2C6010E94082114
:103E80008C179D0708F4BFCFC801DF91CF911F9118
:103E90000F91FF90EF90DF90CF90BF90AF909F90E9
:103EA00008950F931F93CF93DF93EB0183B984E8B9
:103EB00086BF0E94F0208C0106B607FC0EC0CF3FE3
:103EC0008FEFD807C9F30E94F020801B910B8C174D
:103ED0009D0790F38EEF9FEF0BC021B1287F81E00B
:103EE00090E0283211F480E090E09195819591095D
:103EF000DF91CF911F910F9108950F931F93CF934F
:103F0000DF93EC0184EC86BF0E94F0208C0106B6A2
:103F100007FC0EC0CF3F8FEFD807C9F30E94F020F7
:103F2000801B910B8C179D0790F38EEF9FEF02C0C3
:103F300083B190E0DF91CF911F910F9108950F937E
:103F40001F93CF93DF93EC0184E886BF0E94F0209B
:103F50008C0106B607FC0EC0CF3F8FEFD807C9F320
:103F60000E94F020801B910B8C179D0790F38EEF21
:103F70009FEF02C083B190E0DF91CF911F910F912D
:103F80000895CF92DF92EF92FF920F931F93CF93FA
:103F9000DF936B018A017901B9010E94DA1EE60103
:103FA0000C0D1D1DC017D10759F424E926BFDF9160
:103FB000CF911F910F91FF90EF90DF90CF900895D8
:103FC00097FDF3CFB70189910E94511FEBCFCF929C
:103FD000DF92EF92FF920F931F93CF93DF937B01BA
:103FE000EA016901B90181600E94DA1E8701219707
:103FF00098012E193F092C173D0760F497FD14C056
:10400000C6010E947D1F97FD02C0F80180830F5FEB
:104010001F4FEECF97FD08C0C6010E949F1F97FD5E
:1040200003C0CE0DDF1D888324E926BF18161906AC
:1040300014F480E090E0DF91CF911F910F91FF90F9
:10404000EF90DF90CF90089590930F0180930E0131
:1040500008959093ED018093EC010895E091EC01B7
:10406000F091ED01309721F00190F081E02D09945D
:1040700080E00895E091EC01F091ED01309721F09E
:104080000280F381E02D099408952091EA01309196
:10409000EB012817390771F09093EB018093EA0147
:1040A000E091EC01F091ED01309721F00680F7816D
:1040B000E02D099408952091E8013091E901281735
:1040C000390771F09093E9018093E801E091EC01E8
:1040D000F091ED01309721F00084F185E02D0994F5
:1040E0000895FC01329697E080E0915029F02191EB
:1040F0002223D9F38F5FF9CF0895662349F0FC019D
:10410000329608962191621729F0E817F907D1F73E
:1041100080E0089581E008959C01FC0132969FEFB4
:1041200080E04191461789F09F3F19F4411101C089
:10413000982F8F5F8630A9F79F3F39F0F901E90F7B
:10414000F11D97FDFA956283089508959C012A5FF9
:104150003F4FFC014281461301C012820196821733
:104160009307B9F708950C948C200C94A62002961E
:1041700026E0FC0111922A95E9F7089508950C9420
:10418000BE200C94BF200C94BE200C94BE200C9436
:10419000BE20CF930E94C5200E947B040E94C320B2
:1041A000C0E08C2F0E941405892B29F4CF5FC63004
:1041B000C1F780E001C081E0CF910895089580911A
:1041C000F00181110C943F0608950E94F1090C94AE
:1041D00045068BE083BF8BEB8CBF82E089BF0895DF
:1041E0002FB7F8948091B1029091B202A091B302DE
:1041F000B091B4022FBF08952FB7F8946091B10227
:104200007091B2028091B3029091B4022FBF0895D1
:104210009C014FB7F8948091B1029091B202A091A5
:10422000B302B091B4024FBF821B930B08957894F0
:104230001F920F920FB60F9211248F939F93AF93FB
:10424000BF938091B1029091B202A091B302B0915C
:10425000B4020196A11DB11D8093B1029093B202E8
:10426000A093B302B093B402BF91AF919F918F918D
:104270000F900FBE0F901F90189560E081E090E0C6
:104280000E942F259CE088E10FB6F894A89581BD87
:104290000FBE91BDFFCF0E94F0209093EF0180935D
:1042A000EE0108950E9428248B9A80E0815041F00D
:1042B000A895E7EBFBE03197F1F700C00000F6CFDF
:1042C0008B98789408950E9450220E9429202FEB09
:1042D00084ED91E0215080409040E1F700C0000063
:1042E00008958091DC02882389F01092DC020E94FC
:1042F000F0209093EF018093EE018091F0018823EC
:10430000D1F11092F0010E94E52011C08091F001DE
:10431000811111C08091EE019091EF010E9408215E
:10432000069728F081E08093F0010E94DF208091C1
:10433000F001882301F10E94DF200E94C920882318
:1043400039F1F89421B3939A822F8C6081BB92B398
:104350008CE0982792BB3FE54AEE90E03150404018
:104360009040E1F700C0000092B3892782BB21BBD7
:104370009398789408950E9431238091E2028823D3
:1043800029F08091C00284FD0E94BE110C94F72197
:10439000089580918502089508959091F6019813EB
:1043A00007C02091F4013091F50126173707A9F0D5
:1043B0008093F6017093F5016093F4018093F1010D
:1043C0007093F3016093F2018091F90284FF05C0BC
:1043D00063E081EF91E00C942D230895BC0184E00B
:1043E0000C94CD21BC0183E00C94CD210895CF9392
:1043F000DF93CAE0D0E08091C00284FF18C08091B2
:104400000202909103029817E1F028E0829FC00118
:10441000112468E08C5F9D4F0E9429238091020245
:1044200090E001968F709927809302020AC00E9443
:10443000312387EB9BE00197F1F700C00000219743
:10444000D1F6DF91CF910895CF93DF93EC01A09146
:104450000302B0E0CD0101968F70992720910202EE
:10446000281779F093E0AA0FBB1F9A95E1F7AC5F8C
:10447000BD4F98E0FE0101900D929A95E1F780936F
:1044800003020E9431230E94F72188E0FE01AAEF77
:10449000B1E001900D928A95E1F7DF91CF910895F7
:1044A00089E790E00895FC01808180768032A1F553
:1044B0008181813061F484819581892B69F58AEF4E
:1044C00091E09093DE028093DD0288E008958230CF
:1044D00041F484E892E09093DE028093DD0281E073
:1044E00008958A3021F483818093840215C0893035
:1044F00099F4828193818115924081F48481958120
:10450000892B61F481E08093F901868197819093F2
:10451000F8018093F70102C080E008958FEF0895BD
:104520002091F7013091F801232B71F02091F901CE
:10453000213051F4FC018081809385021092F801B2
:104540001092F70181E008958FEF08950895FC011E
:1045500093819330D9F068F4913081F0923009F072
:1045600054C08FE994E09093DE028093DD028BE3E8
:104570000895913221F1923291F147C08AED94E091
:104580009093DE028093DD0282E108958281813082
:1045900071F028F08230C9F58CEE94E00AC084E016
:1045A00095E09093DE028093DD0284E0089588EF29
:1045B00094E09093DE028093DD028AE00895828188
:1045C000882329F0813009F58AEC94E002C081EB60
:1045D00094E09093DE028093DD0289E00895848167
:1045E0009581009751F0019781F488E095E09093D0
:1045F000DE028093DD0282E308958AE395E09093E2
:10460000DE028093DD0280E4089580E008951F9328
:10461000CF93DF93162FEA01288124FF05C039814B
:1046200028E82327298302C02AE52883212FFC01BB
:10463000CE010296DC0131913D9321501216DCF33C
:10464000612F0E94F1021C5F1883DF91CF911F91AF
:10465000089540EC52E00C94072349EF52E00C948B
:104660000723CF93DF936091DF02635067FD93C010
:104670008091DB02CCE0D0E0C81BD109CD51DD4FE9
:104680008091DA02803120F4CE010E94A62281C0FE
:104690008D3209F06EC0683009F07BC083EC8093E6
:1046A000B5028AE5809386001092D90288818076CF
:1046B00021F0CE010E94532249C09A811092BE027D
:1046C0008981811106C01092BF022EEB32E082E098
:1046D00038C0853019F49093E00230C08630A1F4E0
:1046E0008B81813041F0823031F0833021F0813292
:1046F00011F0823221F4CE010E94A72201C080E095
:1047000090E49093D90222C0883089F0893019F45E
:104710009093E20213C08A3069F08B3079F48BE415
:104720008093C1028093FA028093CD0207C022EEEB
:1047300032E002C02EEB32E081E003C02EEB32E02B
:1047400080E03093DE022093DD0209C08F3F39F410
:10475000988197FD8E8190E89093D90207C09F8140
:10476000911104C09E81981708F4892F80938500C9
:1047700010C08091D90287FF0CC0CE010E94902208
:104780008F3F21F48EE18093860003C08111109247
:1047900085001092DF028091860084FF4CC08091DA
:1047A00085008F3F09F447C0C82F893008F0C8E062
:1047B0008C1B809385009091B50288E889278093AF
:1047C000B502CC2359F18091DD029091DE02209157
:1047D000D90226FF12C0A5EBB2E02C2FAC01455B3D
:1047E0005240FA01EA0FFB1FE4911196EC931197E6
:1047F000215011962111F5CF08C0E6EBF2E0DC0163
:104800002C2F3D9131932150E1F701962FEF2C0F82
:10481000820F911D9093DE028093DD026C2F86EB58
:1048200092E00E94F102CC5FCC3019F08FEF8093C0
:104830008500C093860084E190B39C7031F4815070
:10484000D9F71092E0021092D802DF91CF9108952B
:10485000CF93DF9385B7886085BF8BB780688BBFA8
:10486000C0ECD2E08BE48983A9EFB2E011968C937F
:104870001197ECECF2E081838AE588838C93808346
:10488000DF91CF91089587FB082E062687FD81953D
:1048900067FD61950E94D2240EF4919507FC8195E5
:1048A0000895AA1BBB1B51E107C0AA1FBB1FA61777
:1048B000B70710F0A61BB70B881F991F5A95A9F7C9
:1048C00080959095BC01CD01089597FB072E16F4B5
:1048D000009407D077FD09D00E94512407FC05D031
:1048E0003EF4909581959F4F0895709561957F4F07
:1048F0000895A1E21A2EAA1BBB1BFD010DC0AA1F21
:10490000BB1FEE1FFF1FA217B307E407F50720F038
:10491000A21BB30BE40BF50B661F771F881F991FB3
:104920001A9469F760957095809590959B01AC01FC
:10493000BD01CF010895EE0FFF1F0590F491E02D0A
:1049400009940E94A924332312F48A1B9B0B0C9414
:10495000BA24A29FB001B39FC001A39F700D811D17
:104960001124911DB29F700D811D1124911D089578
:104970000E94A924B7FF0895821B930B08950E94FB
:10498000A924A59F900DB49F900DA49F800D911D0B
:1049900011240895B7FF0C94BF240E94BF24821BEA
:1049A000930B0895991B79E004C0991F961708F09E
:1049B000961B881F7A95C9F780950895FC01415090
:1049C000504030F001900616D1F73197CF0108958D
:1049D000882799270895FB01DC0104C08D9101907F
:1049E000801921F441505040C8F7881B990B089555
:1049F000E199FECF9FBB8EBBE09A99278DB30895B6
:104A0000A6E1B0E044E050E00C943E25A8E1B0E01F
:104A100042E050E00C943E25262FE199FECF9FBB4B
:104A20008EBBE09A01970DB2021631F02DBB0FB686
:104A3000F894E29AE19A0FBE08950396272F0E94F8
:104A40000D250E940C25252F0E940D25242F0C9446
:104A50000D250196272F0E940D250C940C25262F3D
:104A6000E199FECF9FBB8EBB2DBB0FB6F894E29AA7
:104A7000E19A0FBE01960895DC01CB01FC01E1999A
:104A8000FECF06C0FFBBEEBBE09A31960DB20D9291
:0C4A900041505040B8F70895F894FFCF53
:104A9C00FFFFC800B201010102000C000C0C01194F
:104AAC001A1B1C1D1E1F202122C9212422F621F2B3
:104ABC0021EE21CC21FF5AE200E900EA00B500B654
:104ACC0000B700CD008301CC008A01920194012132
:104ADC0002230224022502260227022A02B300B472
:104AEC00006F007000818283E200E900EA00B500EB
:104AFC00B600B700CD008301CC008A01920194016D
:104B0C002102230224022502260227022A02B300D4
:104B1C00B4006F0070008182830001020202020661
:104B2C0006060909090909090F0F0F0F0F0F1515B3
:0E4B3C001518191919191919191919192324FD
:00000001FF
